:0200000480007A
:100000009710000093800000171100001301810277
:1000100083A10000138211009382F17F1383F1FF0B
:1000200093830100138401802320310023224100A7
:10003000232451002326610023287100232A8100F4
:1000400097100000938040FC17110000130101007D
:1000500003A40000930414001305F47F9305F4FF38
:1000600013060400930604802320810023229100BC
:100070002324A1002326B1002328C100232AD10074
:1000800097100000938080F817110000130181FD84
:1000900083A60000138716009387F67F1388F6FF68
:1000A00093880600138906802320D1002322E100D3
:1000B0002324F1002326010123281101232A2101F1
:1000C000971000009380C0F417110000130101FB8A
:1000D00003A9000093091900130AF97F930AF9FF95
:1000E000130B0900930B09802320210123223101E6
:1000F000232441012326510123286101232A710170
:1001000097100000938000F117110000130181F88F
:1001100083AB0000138C1B00938CFB7F138DFBFFC4
:10012000938D0B00138E0B802320710123228101FC
:10013000232491012326A1012328B101232AC101EF
:10014000171D0000130D4DED971D0000938D0DF64A
:10015000032E0D00930E1E00138F1E00930F1F0021
:1001600093801F00138110009301110023A0CD0183
:1001700023A2DD0123A4ED0123A6FD0123A81D0078
:1001800023AA2D0023AC3D0097100000938000E9C6
:1001900017110000130141F383A200001380120025
:1001A0002320010097100000938080E717110000C2
:1001B0001301C1F183A2000013801200930210000A
:1001C000232001002322510097100000938080E536
:1001D00017110000130101F083A100001382010038
:1001E0009302020013830200130703009307070022
:1001F00013880700930C0800138D0C00930D0D005D
:1002000023203100232241002324A1012326B10110
:1002100017150000130505E297150000938585EC7E
:10022000370610F01306C6F26306B5028326C50032
:100230002320D600832685002320D6008326450070
:100240002320D600832605002320D60013050501B0
:100250006FF09FFD370510F0130505F22320050010
:04026000000000009A
:101000000000000001000000FFFFFFFFFFFFFF7F67
:1010100000000080CDAB00007856341298BADCFE98
:10102000145892360000000000000000000000008C
:10103000FFFFFFFFFFFFFFFFFFFFFFFFFFFFFFFFC0
:10104000FFFFFFFFFFFFFFFFFFFFFFFFFFFFFFFFB0
:10105000FFFFFFFFFFFFFFFFFFFFFFFFFFFFFFFFA0
:10106000FFFFFFFFFFFFFFFFFFFFFFFFFFFFFFFF90
:10107000FFFFFFFFFFFFFFFFFFFFFFFFFFFFFFFF80
:10108000FFFFFFFFFFFFFFFFFFFFFFFFFFFFFFFF70
:10109000FFFFFFFFFFFFFFFFFFFFFFFFFFFFFFFF60
:1010A000FFFFFFFFFFFFFFFFFFFFFFFFFFFFFFFF50
:1010B000FFFFFFFFFFFFFFFFFFFFFFFFFFFFFFFF40
:1010C000FFFFFFFFFFFFFFFFFFFFFFFFFFFFFFFF30
:1010D000FFFFFFFFFFFFFFFFFFFFFFFFFFFFFFFF20
:040000058000000077
:00000001FF
